:020000040000FA
:0400000003303A2867
:08000800A000030EA100831209
:100010008B1C32288B1031181428B11C3228643004
:10002000010203183128182800001628172818285C
:1000300019281A281B281C281D281E281F283110A3
:10004000B114A810031005190314AA0DA90DA80DC9
:10005000B00B322831152A08AF002908AE00280855
:10006000AD00B11081010B11210E8300A00E200EF6
:02007000090085
:0C007400203084008001840A6030040207
:10008000031C3C281230B000A0218316FF239000EF
:10009000831283160C308505870183128501870141
:1000A000073099000030831691009F008312C830FA
:1000B00083168100831231309000003083168C004B
:1000C000831210308B00BC1B6B2885196B286400D1
:1000D000851D6728E921E12181018E018F010B1126
:1000E0008B100B108C018B17832031199920B30BC7
:1000F0008128031085190314B90DF0303902031952
:100100001B210E2274286400311808000B1D080002
:100110000B11B11031141230B000051D94283214A7
:1001200083160113831208003210831601178312FD
:10013000080031110130B7008B13203037078316C8
:100140009B001C141A088312A400A500C030A50649
:100150001030370783169B001C141A088312A30063
:100160000030370783169B001C141A088312A20064
:100170008B17321CC12822090339A200A309A40944
:10018000A50922082D02031D152923082E02031D8F
:10019000152924082F02031D152901303702031DDC
:1001A000D6283D18D6283D143E14B521023037021A
:1001B000031DDF28BD18DF28BD143E14B92103300C
:1001C0003702031DE8283D19E8283D153E14BD21DE
:1001D00004303702031DF128BD19F128BD153E1466
:1001E000C12105303702031DFA283D1AFA283D16B1
:1001F0003E14C52106303702031D0329BD1A032909
:10020000BD163E14C62107303702031D0C293D1BC5
:100210000C293D173E14C72108303702031D15294C
:10022000BD1B1529BD173E14C821B70A053037027A
:10023000031808009C280130B600B300B400B500D4
:10024000B70085018701B1138320B30B5329031035
:1002500085190314B90DF030390203197A29B40B4A
:100260005329013037020319C9210230370203191B
:10027000CD21033037020319D1210430370203198D
:10028000D921053037020319DD2106303702031961
:10029000DE21073037020319DF2108303702031946
:1002A000E0219630B400311D24293111321C5D2922
:1002B0002D090339AD00AE09AF092F1CB1132F1C56
:1002C0002429B11B24292E182429B1178B1320307F
:1002D0003707BB002F08BA008D2110303707BB004D
:1002E0002E08BA008D2100303707BB002D08BA0058
:1002F0008D218B1785018701B70AB60105303702BA
:10030000031C2429E12108003E1C08003E10103087
:10031000BB003D08BA008D2108008B133A088316F4
:100320001C159A003B089B0055309D00AA309D008B
:100330009C1464009C1899291C1183128B170800C7
:10034000831600309B001C141A088312BC0083160D
:1003500010309B001C141A088312BD00FF30D0001F
:10036000D415D515D615D71508000330D204BD1005
:1003700008000330D2043D1008000C30D204BD1137
:1003800008000C30D2043D110800080008000800E5
:1003900008000508023A850008000508013A8500B2
:1003A00008000C308316850083120508203A85006A
:1003B00008000508103A8500080008000800080039
:1003C00008003D08D200031D08000530BD00D20022
:1003D0000800B601B301B4013C1CF129BC01BC14F6
:1003E000F329BC013C143C08B6006400F729F82945
:1003F000F929FA29FB29B41B8514B41F8510B30B06
:10040000F529B40BF5290310B60CB608031DF52920
:100410000030BB003C08BA008D2108008F0803198A
:1004200008008F01D00FAF2AD00A02305205031DF9
:10043000282A541D1E2AD4015416362AD41D232AD4
:10044000D4015416362A541E362AD401D414362A1E
:10045000D41C2D2AD4015415362A541D322AD40115
:10046000D415362A541E362AD401541501305205AB
:10047000031D492A551D3F2AD5015516572AD51D5A
:10048000442AD5015516572A551E572AD501D51489
:10049000572AD51C4E2AD5015515572A551D532AC2
:1004A000D501D515572A551E572AD501551508309F
:1004B000BC180A305205031D6C2A561D622AD6014B
:1004C00056167A2AD61D672AD60156167A2A561E3D
:1004D0007A2AD601D6147A2AD61C712AD601561544
:1004E0007A2A561D762AD601D6157A2A561E7A2AD7
:1004F000D60156150430BC1806305205031D8F2A4C
:10050000571D852AD70157169D2AD71D8A2AD7013C
:1005100057169D2A571E9D2AD701D7149D2AD71CEE
:10052000942AD70157159D2A571D992AD701D71507
:100530009D2A571E9D2AD7015715BC1CA82AD21CDC
:10054000A82AD51CA82A3C30831685008312AC2A21
:100550000C3083168500831284213D08D200500898
:10056000D1000C305405031D85100C305505031DBA
:1005700005100C305605031D85120C305705031D60
:10058000051251080E020318D92A12305405031D12
:10059000851412305505031D051412305605031D30
:1005A000851612305705031D0516FF30500203193A
:1005B00008008F08031D0800832051080E02031C49
:1005C000D92A18305405031D851006305405031D23
:1005D000851418305505031D051006305505031DFB
:1005E000051418305605031D851206305605031DE7
:1005F000851618305705031D051206305705031DD3
:0406000005160800D3
:084000000200030006000400A9
:02400E00CC01E3
:10420000010003000300030003000200020002009B
:1042100002000000000000000000FF00FF00FF009F
:10422000000000000000000000000000000000008E
:104230000000C000C000C000C000FF00FF00FF0081
:104240000100C300F300CF00FF00C300F300CF0064
:10425000FF00C300F300CF00FF00FF00FF00FF00DE
:10426000FF00FF00FF00FF00FF00FF00FF00FF0056
:10427000FF00FF00FF00FF00FF00FF00FF00FF0046
:10428000FF00FF00FF00FF00FF00FF00FF00FF0036
:10429000FF00FF00FF00FF00FF00FF00FF00FF0026
:1042A000FF00FF00FF00FF00FF00FF00FF00FF0016
:1042B000FF00FF00FF00FF00FF00FF00FF00FF0006
:1042C000FF00FF00FF00FF00FF00FF00FF00FF00F6
:1042D000FF00FF00FF00FF00FF00FF00FF00FF00E6
:1042E000FF00FF00FF00FF00FF00FF00FF00FF00D6
:1042F000FF00FF00FF00FF00FF00FF00FF00AA001B
:00000001FF
